:060000000C94BD000C94FD
:1000060000000C9400000C9474050C9400000C94F1
:1000160000000C9400000C9400000C9400000C945A
:1000260000000C9400000C9400000C9400000C944A
:1000360000000C94A7050C94C7050C94F5050C94C8
:1000460000000C9400000C9400000C9400000C942A
:1000560000000C9400000C9400000C9400000C941A
:1000660000003F065B4F666D7D077F6F777C395ECC
:100076007971140001000173505814050107013EFF
:10008600775814100103013E0000140314050130D3
:1000960000001400010001735C1C14000100010043
:1000A600777414171906013E045414101404013011
:1000B600587414000100016D79393C000100014FAC
:1000C60077733C00010001785C1C3C000100017163
:1000D6003E3860047E049C04B004C404D804F604CC
:1000E60014053205500578050306090102030406C6
:1000F600080A050A38CF0738876638068677060065
:10010600775B00774F00776600777D00777F007713
:10011600063F737D0073065B00001C0C480DAC0D9A
:10012600DE0D100E560EA60E000F5A0FBE0F04104F
:10013600B80ABD0B140C3F0C6B0CA70CED0C3B0D59
:10014600890DE00D1D0E200001002D4E414E004987
:100156004E460000020002001E01160000032001A8
:1001660016001603360101009E034C010100C2036E
:100176004E010000F894EE27EFBBF1E0F5BFE5BFB6
:10018600F8E1A895A4B7A77FA4BFF0936000E09319
:1001960060008DE0A2E0BB27ED938A95E9F780E049
:1001A60098E0A0E0B1E0ED930197E9F7EAE5F1E028
:1001B60085919591009761F0A591B591059015905F
:1001C600BF01F00105900D920197E1F7FB01F0CF19
:1001D600E0E0EEBBEFEFEDBFE8E0EEBFC0E0D3E05E
:1001E6000C947006AA93E8810E94310C3396E49130
:1001F600EF70E06C0E94370CE0917A00E071E1F359
:100206000E943F0C21960895E8EC0E94370CE0917D
:100216007A00E071E1F30E943F0CE151F1400F01D9
:10022600AEE2B0E00E947D0FF0E0E7FDFFEFE00DEB
:10023600F11D08951A9310E01C3098F4A5E01A9F5A
:10024600F0010E94490CA5E01A9FF001E45DFC4F05
:10025600A0E0A083A5E01A9FF0010E94500C1F5F4A
:10026600EBCFE2E07E2EF1980E94570C6624E0E088
:10027600E0938903E0938A030E945D0CE0E0E0933B
:100286009703E4E6E0939803E89422F821F80E94A5
:10029600640C0E94690CAFEF0E949C0EE0FB27F8ED
:1002A600E89426F8F49AF39AF29A30F844240E94D5
:1002B6006E0CE0E0E0939F03E093A003E093A103BC
:1002C600E093A203E093A303E093A403E093A503C2
:1002D600E093A6030E94740CE03011F0E93C08F0AC
:1002E60003C00E94740C01C0E2E3E093AD03E0EBAF
:1002F600F3E0FA93EA93E0E0EA93A2E1B0E00E9429
:10030600210C0E94790CEF3FAFEFFA0731F4A5E319
:10031600B0E0E1E7F2E70E94890F0E94790CDF0165
:10032600ECE3F0E00E94DD0EE093AE03F093AF0342
:1003360010E01930C8F40E947E0CAE0FBF1F0E9459
:100346007D0FEF3F79F40E947E0CAE0FBF1FE12FA9
:100356000E94910F0E947E0CAE0FBF1F1196E0E027
:100366000E94910F1F5FE5CFAEE2B0E00E947D0FC5
:10037600EF3F29F4AEE2B0E0E2ED0E94910F15C224
:10038600AA93E881A0918703EA1711F4E0E801C077
:10039600E0E026C40E94740F1A930A9310E000E06E
:1003A6000E94850CA935EEE3BE07EFE08E07E0E07C
:1003B6009E073CF0E6E8E0938403E0E80E948A0C9E
:1003C6008FC00E94850CAD39EFEFBE07EFEF8E07A9
:1003D600EFEF9E074CF4E6E8E0938603E0E8E0934F
:1003E6008403E09385037CC0AD81AA234AF401E02F
:1003F600EA81FB816C817D810E94670E0E948F0CD1
:10040600EFEFE09387030E94850CA73EE3E0BE076B
:10041600E0E08E07E0E09E077CF00E94940C0E94CC
:100426001A0F1E2F0E94940C0E949A0CE0918703CB
:10043600EF5FE0938703E7CFA12FE5E00E94A10ECF
:100446000E94850CFF27662777270E949D0C0E9435
:10045600A00C0E94150F0E94A20F49F0E859FF4F09
:10046600E491EF93A0E08CDFAF91EA2B01C0E0E0CE
:10047600E09384030E94A00C0E941A0F0E948F0C26
:10048600E0918403E03039F40E94940C0E94150F29
:100496000E94A20F69F00E94940C0E94150FE85961
:1004A600FF4FE491EF93A1E06BDFAF91EA2B01C020
:1004B600E0E0E0938503003029F0E0918403E064F6
:1004C600E09384030E94940C0E941A0FE859FF4F90
:1004D600E491EF93A2E054DFAF91EA2BE093860319
:1004E6001981088126960895BA93AA931A930E94B1
:1004F600A60CE15DFC4FA5E0B0E0A083B1830E94AD
:10050600AB0CA981BA810E944F0F0E161F0620F46C
:100516000E94A60C0E94500C11E01B30D0F40E94E1
:10052600AB0CE12FA981BA810E94B40C0E944F0F37
:100536000E161F0660F00E94A60CE15DFC4FBF017F
:10054600AAE01A9FF001DB01F0E0ED93FC931F5F38
:10055600E4CFEB81E030C1F40E94A60CE15DFC4FD4
:10056600FF93EF9360817181A0915203B091530381
:10057600E8ECF0E00E94DD0EDF01FB01EA1BFB0B5D
:10058600AF91BF91ED93FC9318811BC31A932297E9
:10059600EEE30E94BA0CE0E0E883E983A881B98122
:1005A6001F9750F40E94C30C1C9903C01C9BFECFDE
:1005B60003C00E94C70CF2CF22960E94740C0E94C0
:1005C600CD0C0E94D50C29F10E94DE0C49F00E9448
:1005D600E60C1E9902C0F29801C0F29AF29B1F5FC8
:1005E6000E94ED0C49F00E94E60C1F9902C0F39898
:1005F60001C0F39AF39B1150113010F0193C08F02A
:1006060012E30E94F50C1C9903C01C9BFECF01C08F
:10061600D8CF0E94740CEF3F11F4123311F0E1179A
:1006260009F413C0AFE2B0E00E94FF0CA881B981C3
:100636001F9750F40E94C30C1C9903C01C9BFECF4D
:1006460003C00E94C70CF2CF2296AFC01A9322971E
:10065600E0E30E94100DA881B9811F9750F40E9413
:10066600C30C1C9903C01C9BFECF03C00E94C70C81
:10067600F2CF22960E941C0D0E94CD0C0E94D50C32
:1006860001F10E94DE0C49F00E94E60C1E9902C0A0
:10069600F29801C0F29AF29B1F5F0E94ED0C49F09E
:1006A6000E94E60C1F9902C0F39801C0F39AF39BCF
:1006B60011500E94F50C1C9903C01C9BFECF01C073
:1006C600DDCF0E941C0DE11799F0A3E3B0E00E9474
:1006D600FF0CA881B9811F9750F40E94C30C1C9986
:1006E60003C01C9BFECF03C00E94C70CF2CF22960C
:1006F6005CC01A932297E8E70E94100DA881B98181
:100706001F9750F40E94C30C1C9903C01C9BFECF7C
:1007160003C00E94C70CF2CF22960E94210D0E94B0
:10072600CD0C0E94D50C29F10E94DE0C49F00E94E6
:10073600E60C1E9902C0F29801C0F29AF29B1F5F66
:100746000E94ED0C49F00E94E60C1F9902C0F39836
:1007560001C0F39AF39B1150113010F0133008F0DA
:1007660011E00E94F50C1C9903C01C9BFECF01C032
:10077600D8CF0E94210DEF3F11F4113011F0E1178F
:1007860009F413C0A4E3B0E00E94FF0CA881B9816C
:100796001F9750F40E94C30C1C9903C01C9BFECFEC
:1007A60003C00E94C70CF2CF2296199108951A939E
:1007B6000A930E94260DE9E7E0938503E8E70E9485
:1007C6002B0DA881B9811F9750F40E94C30C1C9968
:1007D60003C01C9BFECF03C00E94C70CF2CF22961B
:1007E60000E00E94310DEF3F11F000E801C000E08B
:1007F6000E94360DA881B9811F9750F40E94C30C40
:100806001C9903C01C9BFECF03C00E94C70CF2CFED
:1008160022961E9918C0E0E3F0E00F010E94310D08
:100826000E94420D0E94360DA881B9811F9750F48F
:100836000E94C30C1C9903C01C9BFECF03C00E94E0
:10084600C70CF2CF229600E00E94690CEF3F09F038
:1008560000E80E94480DA881B9811F9750F40E94B4
:10086600C30C1C9903C01C9BFECF03C00E94C70C7F
:10087600F2CF22961E9932C0E1E3F0E00F010E940A
:10088600690C0E94420D0E94480DA881B9811F97EC
:1008960050F40E94C30C1C9903C01C9BFECF03C0DE
:1008A6000E94C70CF2CF22960E94260D0E94540D7C
:1008B600A881B9811F9750F40E94C30C1C9903C0EC
:1008C6001C9BFECF03C00E94C70CF2CF22960E944B
:1008D600690CAFEF0E949C0EE0FB27F800E00E9437
:1008E600590DEF3F09F000E80E945E0DA881B9811D
:1008F6001F9750F40E94C30C1C9903C01C9BFECF8B
:1009060003C00E94C70CF2CF22961E992BC0E2E3C9
:10091600F0E00F010E94590D0E94420D0E945E0DEB
:10092600A881B9811F9750F40E94C30C1C9903C07B
:100936001C9BFECF03C00E94C70CF2CF22960E94DA
:10094600260D0E94540DA881B9811F9750F40E946C
:10095600C30C1C9903C01C9BFECF03C00E94C70C8E
:10096600F2CF229613DE72DEC4DE10E0173008F0F6
:10097600B5C0103009F4B0C0143009F4ADC02297E8
:10098600E12F0E94310C3596049000928403E12FEA
:100996000E94310C3696049000928503E12F0E9446
:1009A600310C3796049000928603E0E0E883E983F1
:1009B600A881B9811F9750F40E94C30C1C9903C0EB
:1009C6001C9BFECF03C00E94C70CF2CF2296A4E068
:1009D600B0E0E12F0E94B40C0E946A0DE8EEF3E04D
:1009E6000E94710D0E94D50C09F43FC00E94DE0CD6
:1009F60069F00E94E60C1E9902C0F29801C0F29AB4
:100A0600F29904C0ABEAB3E00E94760D0E94ED0CA9
:100A160069F00E94E60C1F9902C0F39801C0F39A90
:100A2600F39904C0ABEAB3E00E947C0D0E94820DEC
:100A3600A83EE3E0BE0730F00E94820DA13BE4E051
:100A4600BE0710F00E94870D0E948E0DE85EF340EF
:100A56000E94930D9FDCA1E0B0E00E944F0E1C990E
:100A660003C01C9BFECF01C0BDCFA4E0B0E0E12FC8
:100A76000E94B40C0E94790F0F01EF3FAFEFFA0707
:100A860031F40E94820DAC34E4E0BE0729F00E94E6
:100A9600820D0A161B0609F41FC0A4E0B0E0E12F80
:100AA600F0E0EE0FFF1FAE0FBF1F0E948E0D0E94DB
:100AB600890F0E94260D0E94540DA881B9811F97A7
:100AC60050F40E94C30C1C9903C01C9BFECF03C0AC
:100AD6000E94C70CF2CF22961F5F48CF0991199149
:100AE60008950E94980D1E9B0AC01F9B08C0A091E6
:100AF6009A03B0919B03A033E5E7BE0711F40E9469
:100B06009F0DA0E01D99A1E0E0E031FCE1E0EA17CD
:100B160031F00E949F0DE8941D99689431F80E9467
:100B2600A60D2BC0E0E0E4BDE2E0E5BDE0919E034A
:100B3600E7BDE0916E00E260E0936E00E0916E002A
:100B4600E160E0936E0008950E94980D27FC0AC0AC
:100B560026FC08C0AAE9B3E00E94760DE133A5E7BA
:100B6600FA0758F0E0E3F5E7E0939A03F0939B0366
:100B7600299A2A9A2B9AE0E0EBB9E991EFBFF9910D
:100B8600E991B991A991189518950E94740F0E9440
:100B9600AC0DE055FC4F0F010E946F0F0E94B10D86
:100BA6000E94590ED0010E945E0F0E94AC0DEB54BC
:100BB600FC4FA0E0A0830E94AC0DEC54FC4FA1E0DA
:100BC600A08325960895AA930E94BA0DE081E0308D
:100BD60031F00E94BA0DA0E0A083E1E001C0E0E0A0
:100BE600219608950A921A926A937A938A939A930F
:100BF600AA93BA93EA93FA93EFB7EA931A93299AC8
:100C06002A9A2B9AE0E0EBB9E0918803F0E0EC57E2
:100C1600FC4FE081EBB9E5B1EE60E5B915B0E091C6
:100C26008803EF5FA1E00E946F0EE095E121E5B930
:100C3600F09B07C00E94B10DE6E00E94770EE770B8
:100C460009F001C05F9AA0918803AF5FA093880363
:100C5600A33018F0E0E0E0938803AFE9B3E00E9428
:100C6600590FEF5FFF4F6F4F7F4F0E94630F10E0EA
:100C7600133028F5A6E01A9FF001DF01EC54FC4F73
:100C8600E081E03059F0FD01E055FC4FDF010E94A4
:100C9600530F0E94B10D0E94A60F09F00EC0A6E0E8
:100CA6001A9FF001EB54FC4FA1E0A083A6E01A9F27
:100CB600F001EC54FC4FA0E0A0831F5FD9CF19913F
:100CC600E991EFBFF991E991B991A991999189912A
:100CD6007991699119900990189520E033E0AADA84
:100CE600EFE0E4B9EEEFE5B9E7E0E7B9E0E0E8B94F
:100CF600EBB9EFEFEAB9E7E8E0937A00E0ECE093CE
:100D06007C00E8E3E0937E0041982898429840985A
:100D1600E5E0E3BFF894E0E0E0936900EDBBE1E0D5
:100D2600E0936800E0EFE0936B00E1E0EBBB7894C2
:100D3600F9DE1F9902C01E9B01C038C01AE0E12FE0
:100D46001150E03099F1E12FF0E0E859FF4FE491BE
:100D56000E948A0C0E94C10D1F9902C01E9B01C0F1
:100D660025C0103011F5E0E40E948A0C0E94C10DE6
:100D760010E0A12FE9E40E94C70D4CF4A12FB0E0CA
:100D8600A7FDBFEFEFEF0E94910F1F5FF2CFE9E3E0
:100D9600E0938403E8E3E0938503E0E5E0938603CC
:100DA600ACEDB5E00E944F0E01C0C9CF1E9BFFDC23
:100DB6000E94590DEF3F11F026E133E0E0E0E093A9
:100DC6008D03E0938E035524E093A703E093A803D5
:100DD600E093A903E093AA03A5E0B0E080E090E0E9
:100DE600D9DAECE9E0938403A8EEB3E00E944F0E53
:100DF600A8EEB3E0BA93AA9324971A930A9300E055
:100E060010E0E0E0EA83EB83EC83ED830233E0E07D
:100E16001E0754F4F9D90E94850C0E94970E0E9471
:100E26009D0C0F5F1F4FF2CF0E94850CE2E3F0E0AE
:100E360060E070E00E949A0C0E94850CABDA0E947A
:100E4600850CA436E0E0BE07E0E08E07E0E09E07F2
:100E56001CF4AD81AA230AF403C0E8E7E0938403F7
:100E6600AE81BF810E944F0E198108812896F099A4
:100E760008C0ACE9B3E00E94760DE739A0E0FA07B6
:100E860008F451C0E0E0EBB929982A982B98EAB902
:100E9600EBB98895E89432F81C9904C0ACE9B3E044
:100EA6000E947C0D1CEFE1E8F0E0E4911E17B4F41B
:100EB600103031F4E4E3F3E0A0E0B0E0A083B183C6
:100EC600A1E090D9A0913403B0913503EA0FFB1F3E
:100ED600E0933403F09335031F5FE5CFE0913403CD
:100EE600F091350366277727ACE4B4E080E090E024
:100EF6000E94CE0D0E94D30DE0933403F093350388
:100F06000E94DA0DA0912F03B0913003882799270C
:100F160041DAE3E7E0938403EFEFEAB91E9B02C0F0
:100F26001F9901C0FBCFF09B65C0A0919803AA3022
:100F3600A8F00E94E10D80F0ABE8B3E00E94760DC8
:100F4600A0918B03B0918C03509728F00E94570C08
:100F5600E0E0E093980302C00E94570CE0919803EA
:100F6600E03039F4289AE1E0E0939803E0E0E0937A
:100F76009903A0919803A13081F4A0919903A5301B
:100F860030F4E0919903EF5FE093990306C0E0E047
:100F9600E0939903E2E0E0939803A0919803A230CE
:100FA60059F40E94E10D28F0F19A5524289AE4E6B6
:100FB60001C0E3E0E0939803A0919803A33039F4CD
:100FC600E0E0E09399032898E4E0E0939803A09189
:100FD6009803A43079F4A0919903A83230F4E091F3
:100FE6009903EF5FE093990305C0E0E0E09399036E
:100FF600E09398030E94EC0D88279927E0913E0321
:10100600F0913F03662777270E94CE0DE8EEF3E0C6
:1010160060E070E00E94F00EE0934303F093440317
:101026000E94DA0D6624ECE06E1608F0B9C3E62DD0
:101036000E94310C3196E491E03009F4AFC3F59B80
:1010460005C0A2E8B3E00E94760D05C0E0E0E0939B
:101056008203E0938303E72D0E94310CE491A09173
:101066008203B0918303F0E0AE17BF0760F0F598F6
:10107600E9E0E71541F4E0919703E03021F4F69AB0
:10108600E1E0E0939703F69B05C0A1E9B3E00E9477
:10109600760D02C00E94F10DA0919103B0919203CA
:1010A600A036E0E0BE07C0F0ECEEF0E00E946C0F68
:1010B600E0919703E150F0E0E251FF4FE491FF2702
:1010C600662777270E94D30EE0938F03F093900351
:1010D600F79AF6980E94F10DF79B05C0A3E9B3E0D5
:1010E6000E94760D02C00E94F70DA0919303B09165
:1010F6009403A036E0E0BE07F0F110E01B3074F573
:10110600E12FA8E6B3E0F0E0EE0FFF1FEA0FFB1FAA
:10111600FF93EF93E12FA8EDB0E0F0E0EE0FFF1F95
:10112600EA0FFB1F0E946C0F88279927E0918F0317
:10113600F0919003662777270E94D80EDF01CB0136
:10114600ECEEF0E00E94680F662777270E94150FE5
:10115600AF91BF91ED93FC931F5FD0CFF798689442
:1011660020F8E8E7E0938403E0E00E948A0CA4EF0D
:10117600B1E00E944F0E20FE05C0A5E9B3E00E9433
:10118600760D02C00E94FD0DA0919503B0919603C5
:10119600A036E0E0BE0780F0E0E0EA930E94790C1A
:1011A600662777270E94030E882799270E94CE0D6F
:1011B600ECDCE89420F8F09AA4E0B0E0E62D0E947A
:1011C600B40C0E946A0D0E94820DA83EE3E0BE07A1
:1011D60030F00E94820DA13BE4E0BE0710F00E94B1
:1011E600870D10E0E62D0E94310C3196E491EC5FFC
:1011F600A12F0E94C70D0CF0D1C2A62D0E94F500AA
:10120600E0938003F09381030E94080EDF01EC91C6
:10121600EF5FEC930E94080EA081A53088F00E9433
:101226000F0EE35DFC4F0F01DF010E944F0FA091EF
:101236008003B0918103EA0FFB1FD001ED93FC936D
:101246000E94080EA081E62D0E94310C3196E49191
:10125600EC5FAE1708F44FC00E940F0EDF01E15D90
:10126600FC4FFF93EF93A35DBC4F0E944F0F662781
:101276007727DF01CB010E948E0D662777270E9414
:10128600CE0D0E94D30DAF91BF91ED93FC930E94BA
:10129600310DEF3FC1F40E940F0E0E94140E3296DC
:1012A600E491F0E00E94DD0EDB01ED93FC930E94D9
:1012B6000F0E0E94140E3296E491F0E00E94AB0EDF
:1012C600DB01ED93FC930E94080EA0E0A0830E9430
:1012D6000F0E0E94490CA0918003B0918103AF3F8D
:1012E600E3E0BE0741F40E940F0EE15DFC4FAFEF55
:1012F600BFEFA083B1831E9B05C0A39409F4AA94F3
:1013060099240DC0939409F49A94AA24F29B07C0D9
:1013160099241F9902C0689421F8689424F81F9BA9
:1013260005C0D39409F4DA9488240DC0839409F493
:101336008A94DD24F39B07C088241E9902C0689412
:1013460022F8689423F81C9B05C0C39409F4CA9438
:10135600BB2409C0B39409F4BA94CC24F49B03C00B
:10136600BB24689425F81E9902C0F29801C0F29A2F
:101376001F9902C0F39801C0F39A1C9902C0F49811
:1013860001C0F49A22FE43C0A4EFB1E0BA93AA9337
:1013960024971A930A9300E010E0E0E0EA83EB83D7
:1013A600EC83ED830233E0E01E075CF40E94070144
:1013B6000E94850C0E94970E0E949D0C0F5F1F4F86
:1013C600F1CF0E94850CE2E3F0E060E070E00E945D
:1013D6009A0C0E94850C0E94CD010E94850CA436B1
:1013E600E0E0BE07E0E08E07E0E09E071CF4AD817A
:1013F600AA230AF403C0E8E7E0938403AE81BF8121
:101406000E944F0E198108812896E89422F821FE41
:101416001AC0E89421F822F8E0E50E94BA0C1E9B57
:1014260002C01F9901C0FBCFF09841982898F69802
:10143600F798E89420F8E0E0E0938D03E0938E03BC
:101446000E941D01BBCC1D9902C0F09B01C023C0A8
:101456000E941C0DA0913E03B0913F03F0E0AE1731
:10146600BF0758F4AEE7B3E00E94760D309721F43B
:10147600AEE7B3E00E947C0D02C00E946E0C0E9493
:10148600EC0DA93EE3E0BE0728F0E0E0E0939C0304
:10149600E0939D0302C00E946E0C0E94210DAE2FA8
:1014A600EF3F11F4E1E001C0EA2F0E94910EA1E79F
:1014B600B2E780E090E00E94D80EA0917E03B09142
:1014C6007F03882799270E94A60F34F40E94EC0D0B
:1014D600A93EE3E0BE0708F404C0419A0E946E0CE0
:1014E60001C0419825FE1EC020FE08C0E0E6F0E0DF
:1014F600E0939503F0939603E89425F8F79B08C0CC
:10150600E0E6F0E0E0939303F0939403E89425F883
:10151600F69B08C0E0E6F0E0E0939103F0939203B7
:10152600E89425F825FE17C04394E2E0E41508F494
:101536004424A42DE0E00E94A60EE03011F4429867
:1015460001C0429AA42DE1E00E94A60EE03011F4FB
:10155600409801C0409A24FC07C097FE04C0A1E051
:1015660032DBE03009F446C00E941D0E0EDB0E94FD
:10157600A60DF79B14C00E94F70D0E94260EA138F7
:10158600EEE3BE0758F4E091AD030E94260EF0E0AC
:10159600EA0FFB1FE0938F03F09390032BC020FE0E
:1015A6000EC00E94FD0D0E94030EA538E3E0BE07A3
:1015B60028F40E942B0E35960E94710D1BC0F69BD7
:1015C6000EC0A0919703AC3020F4E0919703EF5F33
:1015D60001C0E1E0E09397030E94F10D0BC0E0E04B
:1015E600E71510F47A9402C0E9E07E2E0E945D0CA5
:1015F6000E94570C23FC07C087FE04C0A1E0E3DA73
:10160600E03009F443C00E941D0EBFDA0E94A60D09
:10161600F79B14C00E94F70D0E94260EA93EE3E038
:10162600BE0758F0E091AD030E94260EF0E0AE1B17
:10163600BF0BA0938F03B093900328C020FE0CC06D
:101646000E94FD0D0E94030E159728F00E942B0E96
:1016560035970E94710D1AC0F69B0EC0A091970394
:10166600A23020F0E0919703E15001C0ECE0E09356
:1016760097030E94F10D0AC0E9E07E1610F47394F8
:1016860001C077240E945D0C0E94570C0E94640CD6
:101696000E942B0E309721F0A0E095DAE03009F495
:1016A60003C0F19AE1E05E2EF19B11C0419A0E94BF
:1016B6005D0CE1E0E51511F4EAE001C0EBE07E2EF9
:1016C600F598E5E07E2EF098E4E6E0939803F59B26
:1016D60011C0E0918803F0E0BF01EC57FC4F0F0109
:1016E600E72D0E94310C3596E60FF71FE491D001E5
:1016F600EC9338C0F69B15C0E0918803F0E0CF016B
:10170600EC57FC4FBF01E0919703E150A3E0EA9F3D
:10171600F001E650FF4FE80FF91FE491DB01EC936F
:1017260021C0F79B05C00E94260E8827992718C05E
:1017360020FE05C00E94030E8827992711C032FE9D
:1017460011C00E94300EEF3FAFEFFA0729F4A0E474
:10175600B2E48FE090E004C00E94300E0E94930D28
:101766000E94CD010E943A0EACE3B0E080E090E02A
:101776000E94B30E7F936F93FF93EF930E94790CB1
:10178600AF91BF918F919F91662777270E94F00EA8
:10179600E0935703F09358031F5F24CD639443CC23
:1017A600689432F830FC04C0A0919803AB3040F046
:1017B600E2E0EA93E9E0EA93A8E6B3E00E94770262
:1017C600A091A303B091A4038091A5039091A603D1
:1017D6000E943A0E0E945E0EA0913E03B0913F0316
:1017E600882799270E94CE0D0E94430E0E94590E0B
:1017F600E093A703F093A8036093A9037093AA0349
:101806000E943A0EE093A303F093A4036093A5030A
:101816007093A6030E94790C66277727ACE3B0E0A5
:1018260080E090E00E94CE0D0E94430E0E94F00ED2
:10183600E0934803F09349031ACBFFCFBA93AA93D8
:10184600B981A881109631F0FC81EB816A816193A0
:101856001197E9F7EB81FC8125960895F0E00E9447
:10186600830EE858FF4F0895E0937C00E0917A00DC
:10187600E064E0937A000895E0917A00E061E093F5
:101886007A00E0917800F09179000895E35DFC4FCD
:10189600A0E0B0E0A083B1830895E15DFC4FA0E035
:1018A600B0E0A083B1830895E0E0E0938B03E0937A
:1018B6008C030895F59AE0E0E0938203E0938303B6
:1018C6000895E89425F824F823F80895A1E3B0E0F4
:1018D6000E947D0F0895E0E0E0937E03E0937F038E
:1018E6000895AFE2B0E00E947D0F0895A5E3B0E051
:1018F6000E94790F0895ACE1B0E0E12FF0E0EE0F21
:10190600FF1F0895AA81BB818C819D810895E09374
:101916008603E09385030895EA83FB836C837D83C6
:101926000895F0DFEAE0F0E060E070E008950E94DC
:10193600150FF2CF0E94590EEFCFE4DFE4E6F0E098
:1019460060E070E00895EB81A5E0EA9FF00108955C
:10195600EC81A5E0EA9FF001E15DFC4F008011807B
:101966000895F0E0EE0FFF1FAE0FBF1F0895E0933E
:101976008403EDE6E0938503E8E7E09386030895A4
:10198600A4E6B0E00C944F0EE881F9813196E88325
:10199600F98308951E2FE8EEF3E0E0938D03F093AC
:1019A6008E030895ADE8B3E0ED91FD913197FE9376
:1019B600EE9330970895A0E01E99A1E0E0E0F29939
:1019C600E1E0EA170895E8E8F3E1E0938D03F09388
:1019D6008E030895A0E01F99A1E0E0E0F399E1E00D
:1019E600EA170895A12FBB27882799270E94CD01C2
:1019F600A1E0B0E00C944F0EE12F0E94910F2297C8
:101A0600EDE6E0938403ECE1E0938503EEE5E093F5
:101A16008603E0E0E883E9830895E0938403ECE538
:101A2600E0938503E1E7E0938603E0E0E883E9835A
:101A36000895A3E3B0E00E947D0F0895A4E3B0E00B
:101A46000E947D0F08952297EDE6E09384030895A2
:101A5600E0938603E0E0E883E9830895A0E3B0E03D
:101A66000E947D0F08952297E02FE065E09384039E
:101A7600E02FE967E0938503E02FED66E9CFE09577
:101A8600D0010E94910F005808952297E02FE86335
:101A9600E0938403E02FED63E0938503E02FE66790
:101AA600D7CFECE1E0938503EEE5D2CFA2E3B0E039
:101AB6000E947D0F08952297E02FE863E093840348
:101AC600E02FE167E0938503E02FE967C1CF0E942D
:101AD600790FE093AB03F093AC030895E0938D0385
:101AE600F0938E030895ED91FD913196FE93EE935A
:101AF6000895ED91FD913197FE93EE930895A0918F
:101B0600AB03B091AC030895ECE4F4E0E093AB03CF
:101B1600F093AC030895E091AB03F091AC03089504
:101B260066277727DF01CB010895AA93BA93EA9334
:101B3600FA93EFB7EA930895EFEFFFEFE0939C0374
:101B4600F0939D030895E0E0E0939A03E0939B03EE
:101B56000895EC81A6E0EA9FF0010895A0919F0305
:101B6600B091A0038091A1039091A2030895E8810A
:101B7600A6E0EA9FF001EB54FC4F0895E09384033E
:101B8600ACEBB2E00C944F0EB0E0A7FDBFEFF0E077
:101B9600AE17BF0708950E94B30EDF01CB0108956B
:101BA600E0E0F4E060E070E00E94F00E0895E1E00D
:101BB600EA93E0E0EA93D9010C947702E0913903C5
:101BC600F0913A03A0918F03B0919003EA17FB07B7
:101BD6000895A0913903B0913A030895E0E0E093A7
:101BE6009103E09392030895E0E0E0939303E0937A
:101BF60094030895E0E0E0939503E0939603089537
:101C0600A0918D03B0918E030895E62DA5E0EA9F7D
:101C1600F001E45DFC4F0895E62DA5E0EA9FF00192
:101C26000895E15DFC4FBF01DF010E944F0FDF0108
:101C3600E62D14CEE1E0EA93E091AE03F091AF0316
:101C46000E948A0E6DCFA0918F03B09190030895E4
:101C5600E0918D03F0918E030895E72DA5E0EA9FAC
:101C6600F001E15DFC4FDF010E944F0F0895E09106
:101C76009F03F091A0036091A1037091A2030895C0
:101C8600E5E00E94770EA091A703B091A80380918A
:101C9600A9039091AA030895109639F08AEF90E06F
:101CA6000197F1F7A8951197C9F70895EA0FFB1F59
:101CB600681F791F0895EA1BFB0B680B790B0895C3
:101CC600F195E195F0400895F09560957095E19550
:101CD600FF4F6F4F7F4F0895EE230E2EEA2F19F018
:101CE600EE0F0A94E9F70895EE230E2EFD01BC01CE
:101CF60031F076956795F795E7950A94D1F70895AB
:101D0600EE0FFF1FEE0FFF1FEE0FFF1F0895F69554
:101D1600E795F695E795F695E7950895FE2FFF0F5B
:101D2600FF0B6F2F7F2F08956F2F660F660B762F91
:101D36000895EA17E1E009F4EE270895AE17E1E009
:101D460008F4EE270895EA17E1E008F0EE27089573
:101D5600FA9FF02DEB9FF00DEA9FE02DF10D08950F
:101D66007A9F702D6B9F700DF89F700DE99F700D17
:101D76006A9F602D710DFB9F600D711DE89F600DC0
:101D8600711D8827FA9FF02D610D781FEB9FF00DCE
:101D9600611D781FEA9FE02DF10D681F781F0895D9
:101DA6005AD0D6DF0EF48CDF089563D0D9DF0EF457
:101DB6008BDF08950024112490E1AA0FBB1F001C9D
:101DC600111C0E1A1F0A18F40E0E1F1E01C0A16068
:101DD6009A9599F7FD01D00108953F934F935F932C
:101DE600002411244427552730E2AA0FBB1F881F61
:101DF600991F001C111C441F551F0E1A1F0A460B63
:101E0600570B28F40E0E1F1E461F571F01C0A16058
:101E16003A9559F7FD01BC01D001CA015F914F9176
:101E26003F91089526D0D9DF0EF44EDF0895E89449
:101E360097FF09C0A095B09580959095AF5FBF4F6D
:101E46008F4F9F4F689477FD3FDFC7DFFD01BC01D1
:101E56000EF43ADF0895E894F7FF02C031DF689484
:101E6600B7FF06C0A095B095119600F8039400FA46
:101E76000895E89477FF02C027DF689497FF0BC0A8
:101E86000024A095B095809590951196801D901D83
:101E960000F8039400FA0895ED91FC9111970895C6
:101EA600ED91FD916D917C9113970895ED91FD91C2
:101EB6006D917D910895ED93FD936D937C930895B7
:101EC6007E936E93FE93EE9308950590F491E02D24
:101ED6000895A591B4910895E881F9816A817B817D
:101EE60008959A938A93BA93AA930895119602D065
:101EF600FE2F1197F999FECFFF93FFB7F894A1BD76
:101F0600B2BDF89AE0B5FFBFFF91089507D01196CC
:101F1600EF93EF2F03D0EF9111970895F99B02C02D
:101F2600A895FCCF9FB7F894A1BDB2BDF89A80B52D
:101F3600E81719F0E0BDFA9AF99A9FBF089530970D
:101F4600604070400895EA17FB076807790708950F
:00000001FF
